:020000020000FC
:10000000BDC01895189518951895189518951895B8
:10001000189518951895189500E002BF02E008BFE2
:1000200008B701FFFDCF1A95B9F7089511E00FEF5A
:10003000F4CF11E00BEFF1CF11E00EECEECF11E0B9
:10004000EBCF14E0E9CF11E000EBE7CF64E0C69A14
:10005000F6DFC698F4DF6A95D1F7089508EF02BF7E
:1000600002E008BF1894089508B701FFFBCF4A9536
:10007000A9F79894089519E11A95F1F7089508EDF4
:1000800002BF02E008BF18940895A89508B701FFC1
:10009000FACF4A95A1F79894089500B3087009F42F
:1000A00027E0007100B30071C1F700B30071E9F3FC
:1000B0000895EBDF81F400B3007169F000B30470C0
:1000C000C1F7E3DF41F400B3007129F070B3072FEB
:1000D0007470B9F3089500270895552738E0E9DFD3
:1000E000002341F05695007609F050683A95B9F72B
:1000F000052F089500E00895552734E0DADF002346
:1001000041F05695007609F058603A95B9F7052FF9
:10011000089500EF089568E0CCDF6A95E9F7089547
:10012000002702BBBADF1AE0AADFE6DF003FD1F307
:100130000870C1F7C69A8E9A8D9AEDDF8E988D98C9
:10014000C6980895C0E0CEBB0DBBF89404E00CBB8C
:1001500006E00CBB7894E199FECF089500E00EBB59
:1001600001E00CBB0DB308950F93C69A65DFC698E6
:1001700066DF65DF0F910A95B9F70895E0E6FF277E
:1001800000E00193EE23E9F70FED0DBF05E003BF9B
:100190000DE00EBD0CE10BBD07E20ABDBC9ABE9A94
:1001A00000E409BF53DF00EC0BBF0FE005BF00C048
:1001B000D5DF0023A9F401E0D7DF002702BB6DDF04
:1001C0009BDF003FE1F30870D1F787DF06340CF4C2
:1001D000F6CF01E0B7DFC69A32DFC69830DFFBCF3B
:1001E0000AE0C2DFC69A2EE09BDF2A9509F0FCCF19
:1001F00000E0A8DFC69A20DFC698CAE020DFCA95D3
:04020000E9F7F8CF53
:00000001FF
